:0800000000008A110A12052814
:06000A000D30FE00013084
:10001000FF0080308A110A12EC208A110A12831222
:100020000313A1007F08A0000F30A2000130A3003D
:10003000831203132008A4002108A500FF30A007A5
:10004000031CA10324082504031995280430220762
:10005000A400A501A50D2308A5072408FE00250876
:10006000FF0080308A110A12EC208A110A128312D2
:100070000313A7007F08A6002208FE002308FF0044
:1000800080308A110A12EC208A110A12831203139B
:10009000A900A5007F08A800A40002302207A40040
:1000A000A501A50D2308A5072408FE002508FF00CB
:1000B00080308A110A12EC208A110A12831203136B
:1000C000A500AB007F08A400AA0083120313260832
:1000D000AA002708AB00FF30A607031CA7032A08C5
:1000E0002B0403198E282808FE002908FF00803001
:1000F0008A110A12D9208A110A1283120313AA0044
:10010000240884008313251883172A088000A80A6E
:100110000319A90AA40A0319A50A6528063083123F
:100120000313A2070318A30A18288A110A12992890
:1001300008008316031386018112811101158114B1
:1001400001142730A7206130A720A12808008312BE
:100150000313AC002C09AD003C30AC07AE01AF017D
:100160000030831203132F02031DB82864302E02BF
:100170000318CF28FF308312031386008312031362
:100180002D08D020831203138601831203132C0839
:10019000D02083120313AE0A0319AF0AB028080057
:1001A0008312031381000B11831203130B1DD42838
:1001B0000800003A0319E028803A0319E7280034C0
:1001C0007E08840083137F188317000808007F08C7
:1001D0008A007E0882000800003A0319F428803A59
:1001E0000319FE28FF0100347E08840083137F1862
:1001F00083170008FF00840A000808008A110A1209
:10020000E720FD00FE0FFF03FF0A8A110A12E72014
:10021000FC007D08FF007C08080001340034153420
:0C02200001343034003401340034003468
:00000001FF
